:0200000480007A
:100000006F00C004732F2034930F8000630AFF0336
:10001000930F90006306FF03930FB0006302FF038A
:10002000170F0080130F0FFE63040F0067000F000F
:10003000732F203463540F006F00400093E19153FD
:10004000171F000023203FFC6FF09FFF732540F136
:1000500063100500970200009382020173905230F2
:10006000735000189702000093820202739052307E
:10007000B70200809382F2FF7390023B9302F0017B
:100080007390023A9702000093828201739052307B
:100090007350203073503030735040309301000063
:1000A00097020000938242F67390523013051000BD
:1000B0001315F501634C05000F00F00F93011000BC
:1000C0009308D0051305000073000000970200801C
:1000D000938242F3638E020073905210B7B2000015
:1000E000938292107390223073232030E39862F44D
:1000F00073500030970200009382420173901234D3
:10010000732540F173002030B70001FF938000F0A9
:1001100013E7F0F0930EF0F0930120006314D71D65
:10012000B710F00F938000FF13E7000FB71EF00F1A
:10013000938E0EFF930130006316D71BB700FF00AC
:100140009380F00F13E7F070B70EFF00938EFE7FE1
:10015000930140006318D719B7F00FF09380F000B7
:1001600013E7000FB7FE0FF0938EFE0F93015000C0
:10017000631AD717B70001FF938000F093E0000FD8
:10018000B70E01FF938E0EFF93016000639CD015A4
:1001900013020000B710F00F938000FF13E7000F69
:1001A000130307001302120093022000E31452FE0F
:1001B000B71EF00F938E0EFF930170006314D313DC
:1001C00013020000B700FF009380F00F13E7F070F8
:1001D0001300000013030700130212009302200013
:1001E000E31252FEB70EFF00938EFE7F9301800054
:1001F000631AD30F13020000B7F00FF09380F000E2
:1002000013E7000F130000001300000013030700A2
:100210001302120093022000E31052FEB7FE0FF00B
:10022000938EFE0F93019000631ED30B1302000008
:10023000B710F00F938000FF13E7000F13021200B6
:1002400093022000E31652FEB71EF00F938E0EFFAE
:100250009301A0006318D70913020000B700FF0044
:100260009380F00F1300000013E7F0F01302120068
:1002700093022000E31452FE930EF0FF9301B000AE
:100280006312D70713020000B7F00FF09380F0005D
:10029000130000001300000013E7000F1302120008
:1002A00093022000E31252FEB7FE0FF0938EFE0F72
:1002B0009301C0006318D7039360000F930E000FE3
:1002C0009301D0006390D003B700FF009380F00F3C
:1002D00013E0F070930E00009301E0006314D0016E
:1002E000631030020F00F00F638001009391110042
:1002F00093E111009308D0051385010073000000FD
:100300000F00F00F930110009308D00513050000B3
:1003100073000000731000C0000000000000000027
:1003200000000000000000000000000000000000CD
:1003300000000000000000000000000000000000BD
:0403400000000000B9
:1010000000000000000000000000000000000000E0
:1010100000000000000000000000000000000000D0
:1010200000000000000000000000000000000000C0
:1010300000000000000000000000000000000000B0
:081040000000000000000000A8
:040000058000000077
:00000001FF
